:10000000012803138316013085000030860000307C
:100010008700803088000030890000309F00031383
:100020008312C1309F000814881408158815AA305F
:1000300086008700C8201C286400C8208814081582
:10004000E42088100811C82008148815E42008103E
:100050008811C82086130710D72006138710D720D1
:100060008617861207140711D72006170612871461
:100070008711D7208616861107150712D720061676
:10008000061187158712D7208615861007160713C5
:10009000D7200615061087168713D7208614071752
:1000A000D7200614871788140815D720D720881062
:1000B0000811D720D72008148815D720D72008107A
:1000C0008811D720D72088140815D720D72088106A
:1000D0000811D720D72008148815D720D72008105A
:1000E0008811D720D72088140815D720D72088104A
:1000F0000811D720D72008148815D720D72008103A
:100100008811C82088140815E42088100811C82018
:1001100008148815E42008108811C82086130710D9
:10012000D72006138710D7208617861207140711C9
:10013000D7200617061287148711D7208616861136
:1001400007150712D7200616061187158712D72024
:100150008615861007160713D72006150610871672
:100160008713D72086140717D7200614871708147B
:10017000881408158815D720D720D720D720081035
:100180008810081188111C281F151F19C528080080
:10019000C4201E08A2000C30A1003C30A000640066
:1001A000A00BD028A10BCD28A20BCB2808006400FF
:1001B000881BEA202830A100FF30A000A00BDE2819
:1001C000A10BDC2864000800FF30A000A00BE6288B
:1001D00064000800FF3086008700081488140815A2
:1001E000881506108713D720D7200816881FF928EE
:1001F000EA280812D720D720D720D720D720D72009
:020200000800F4
:00000001FF
